:020000040000FA
:020000000528D1
:0800080009008316FF3085009A
:1000100086011130870006309F0040309400831223
:100020000030940094168501860107176120C620D0
:100030000030F3204D20AE0803191A28C1302E06D7
:10004000031D472807138130BD2007171130F32007
:100050004D20AE0803192828C2302E06031D47285C
:1000600007138230BD2007172230F3204D20AE0841
:1000700003193628C3302E06031D47280713843082
:10008000BD2007173330F32005308821182844306D
:10009000F3204C285530F3204C28AE01AA20A01C98
:1000A000080001306F212C30AB000230AC0003019E
:1000B000AD00B22001306F217130AB009F20AE0047
:1000C0000800902080307D208030A500071302308A
:1000D000BD200030BD20A7019A302707A8000130BD
:1000E0000318013E8A0028089921BD20A70AA50B04
:1000F0006C28071700307D200800A6000F30AB00E9
:100100002608AD00962001306F210E30AB009F20F5
:10011000E0302D052606031D7E2801306F210800E2
:100120000713C030BD2007179421080007130230C1
:10013000BD202B08BD202D08BD2007170800071380
:100140000330BD202B08BD205A30BD2007172008E2
:10015000AD0008000713A030BD205A30BD2007179E
:100160002008080007130530BD202B08BD202C08EF
:10017000BD202D08BD2007170800A100930083169D
:10018000141CC02883121308A0000800A501A901AF
:100190002508DC302507A80000300318013E8A003E
:1001A0002808DB20E120A50A05302506031DC82804
:1001B00002306F210800820022342C340C340634C3
:1001C0000134AA0001306F21E720E7200800AA0EC1
:1001D0002A080F3929048600861600000000000056
:1001E000000086120800A50029120230E12029161D
:1001F000FF20003A03190800E120A50AF828250885
:1002000009302507A80001300318013E8A0028089C
:100210008200503472346534733473342034533470
:100220006C346134763465342034313420342034F5
:1002300020340034503472346534733473342034D1
:1002400053346C34613476346534203432342034A1
:1002500020342034003450347234653473347334B1
:10026000203453346C346134763465342034333480
:1002700020342034203400342134213421342134FA
:1002800020345034413453345334453444342034CE
:100290002134213421342134003453346534713411
:1002A000753465346E3463346534203465347234A7
:1002B00072346F3472342034203400344334413487
:1002C0004E342034623475347334203465347234DF
:1002D00072346F3472342034203420340034A3005C
:1002E000F630A20000000000000000000000000046
:1002F00000000000000000000000000000000000FE
:10030000000000000000A20B7229A30B7029080056
:10031000A400FA306F21FA306F21FA306F21FA30E1
:100320006F21A40B892908000A30A200A20B96298C
:1003300008008200FF34FF34FF34FF34FF34FF3401
:10034000FF34FF34C1340034FF34FF340C34003444
:1003500080348034C2340034FF34FF34C33400347A
:10036000FF34FF34FF34FF34FF34FF3400340034F3
:1003700080348034FF34FF34FF34FF34FF34E03402
:10038000FF34FF3402349034093403340034003431
:10039000803480340334B134003400340034003409
:1003A00000340034003400340034003400340034AD
:1003B000803480340234B2340034003400340034E9
:1003C000003400340034003400340034003400348D
:1003D000803480340134B3340034003400340034C9
:1003E000003400340034003400340034003400346D
:1003F000803480342034003400340034003400343D
:10040000003400340034003400340034003400344C
:10041000803480342034003400340034003400341C
:10042000003400340034003400340034003400342C
:040430008034803460
:02400E003A3F37
:00000001FF
